:1000000019C070C89CC831C030C02FC02EC02DC0D0
:100010002CC02BC02AC029C028C027C026C025C09C
:1000200024C023C022C021C020C01FC01EC01DC0CC
:100030001CC01BC011241FBECFEFD4E0DEBFCDBF5C
:1000400013E0A0E0B1E0E8EBF1E102C005900D9211
:10005000A83DB107D9F714E0A8EDB3E001C01D92A7
:10006000A43AB107E1F7F6D1A6C8CACFDC0114164D
:10007000150664F4FB01E95CFE4F20E030E08D9151
:1000800081932F5F3F4F42175307C9F70895E7E366
:10009000F1E08FE492E01192E817F907E1F7089593
:1000A000EF92FF921F93CF93DF93EC01162F6623FD
:1000B00009F47BC0A4EFB3E0FD01E40FF11D508112
:1000C000842F8F5FFD01E80FF11D30818F5FFD01EF
:1000D000E80FF11DE0818F5FA80FB11DAC914C5F5F
:1000E000822F99270F2EFEEFEF2EFFEFFF2EF02D20
:1000F000E80EF91E842F9927E816F9060CF455C06E
:10010000852F8D533D535E2F5D53AD5320E064EF3B
:1001100073E020C0FB01E40FF11DB081842F8F5FDD
:10012000FB01E80FF11D30818F5FFB01E80FF11D2E
:1001300050818F5FFB01E80FF11DA0814C5F842F80
:100140009927E816F9068CF18B2F8D533D535D539B
:10015000AD532D5FFE01E20FF11D880F880F932F25
:1001600092959F70892B80831130F9F0822F8F5FD9
:10017000FE01E80FF11D832F8295807F952F9695C4
:100180009695892B808313501F3F79F0822F8E5FC5
:10019000FE01E80FF11D852F8295880F880F807C66
:1001A0008A2B8083112309F0B5CFDF91CF911F9166
:1001B000FF90EF9008958093E1035091E603543649
:1001C00010F01092E5038091E1038D3009F05CC0DE
:1001D0008091E503823009F057C01092E503652F46
:1001E0007727FB01329724EF33E0E20FF31F4081C2
:1001F000CB010197DC01A20FB31F2C918091E90381
:100200009091EA03841B9109821B91099F7090933E
:10021000EA038093E9039C010024220F331F001C92
:10022000220F331F001C232F302D235C2093E80363
:100230008F73382F335C3093E7038081281729F4BC
:100240008C91381711F491E009C08091E3038F5F1E
:100250008093E30385E48093590490E08091E20366
:10026000882309F07EC0992309F47BC081E0809344
:10027000E2035093E403FB01EC50FC4F8DE08083DC
:1002800082E5809359046DC08091E503813031F19E
:10029000813020F0823009F05FC03EC08091E103E0
:1002A000833239F48091E203882319F481E080934A
:1002B000E5038091E1038093F40381E08093E603FA
:1002C0008091E10399279093EA038093E90381E405
:1002D00080935A0488E58093590443C082E0809358
:1002E000E5038091E103E4EFF3E0E50FF11D808386
:1002F000852F8F5F8093E6032091E1038091E903CE
:100300009091EA03820F911D9093EA038093E90391
:1003100082E480935A0425C08091E103E4EFF3E086
:10032000E50FF11D8083543628F4852F8F5F80936D
:10033000E60302C01092E5038091E1032091E903F6
:100340003091EA03280F311D3093EA032093E9032B
:1003500083E480935A0405C01092E50384E48093FB
:100360005A0480910A01882321F481E080930A01D4
:10037000089510920A010895AF92BF92CF92DF9232
:10038000EF92FF920F931F93CF93DF93CDB7DEB71A
:1003900027970FB6F894DEBF0FBECDBF6C017B016F
:1003A000161617060CF045C080E090E09E012F5F06
:1003B0003F4F60E3F901E80FF91F60830196E816EB
:1003C000F906C1F74115510519F187010150104097
:1003D0005E010894A11CB11CFA01CA016AE070E038
:1003E000C3D6AB01D501A00FB11FCB01880F991F58
:1003F0009B01220F331F220F331F220F331F820F47
:10040000931FE81BE05DEC9301501040672B21F730
:1004100020E030E0AE014F5F5F4FFA01E20FF31FC3
:100420008081F60181936F012F5F3F4FE216F30643
:10043000A1F727960FB6F894DEBF0FBECDBFDF91B0
:10044000CF911F910F91FF90EF90DF90CF90BF90D1
:10045000AF900895AF92BF92CF92DF92FF920F9329
:100460001F93CF93DF931092000110920101E1E6F8
:10047000F0E080E88083108280E18BB91AB8109296
:10048000C00088E18093C10086E88093C20010928A
:10049000C50085E18093C40014BC91E095BD15B8FA
:1004A0008EE384B984E58CBD9DBD8AE080936900AC
:1004B00083E08DBB8CBB10926800789488E58093B4
:1004C00058048093590480935A0480935B0480936A
:1004D0005C0480935D041092E2031092DA03D7DD8E
:1004E00045E150E06CE870E08BEB93E0BFDD81E02C
:1004F00080930001FF24F3940F2EFFEECF2EF3E044
:10050000DF2EF02D08E014E00F2EFBEBAF2EF3E012
:10051000BF2EF02D8091C00088232CF4E6ECF0E093
:100520008081808348DE8091DA03893118F4F0926B
:10053000D90306C01092D903833310F01092DA0366
:100540008091E203882331F38091F603843409F02B
:100550005FC12091E40343E062E482E694E0A0DD21
:10056000409174045091750463E070E08CE091E078
:1005700003DF20916E0430916F048091EB03909122
:10058000EC038217930764F4F092DE031092DF030A
:10059000A901481B590B5093DD034093DC0317C09E
:1005A000281739075CF41092DE03F092DF03821BF8
:1005B000930B9093DD038093DC0309C01092DE035C
:1005C0001092DF031092DD031092DC030CC08091C7
:1005D000DC039091DD03CD9730F08CE390E09093B5
:1005E000DD038093DC033093EC032093EB03332390
:1005F0005CF48DE280933001C901809590959093D1
:100600006F0480936E0403C08BE2809330014091AD
:100610006E0450916F0465E070E081E391E0ACDE20
:10062000409176045091770465E070E0C601A4DE45
:100630008091F10380931B018091F20380931C0150
:100640008091F30380931E0180917604909177044A
:100650008B35910534F0009310018036910524F418
:1006600009C01093100106C0009311018536910551
:1006700024F409C01093110106C0009312018A36B8
:10068000910524F409C01093120106C000931301D0
:100690008F36910524F409C01093130106C000930E
:1006A00014018437910524F409C01093140106C085
:1006B000009315018937910524F409C010931501A1
:1006C00006C0009316018E3791054CF4B4C0109308
:1006D0001601109317018E35910524F006C0009382
:1006E000170103C0F092D80302C01092D8032091E2
:1006F00078043091790484E690E0AC01249FC00135
:10070000259F900D349F900D11246FEF70E02CD534
:10071000EB01AB0165E070E0C6012EDE8091F103D4
:1007200080932C018091F20380932D018091F3033B
:1007300080932E01CB30D10530F000932001C531DC
:10074000D10520F409C01093200106C000932101B7
:10075000CF31D10520F409C01093210106C00093C8
:100760002201C932D10520F409C01093220106C02C
:1007700000932301C333D10520F409C01093230152
:1007800006C000932401CD33D10520F409C0109395
:10079000240106C000932501C734D10520F409C007
:1007A0001093250106C000932601C135D10520F420
:1007B00006C01093260103C00093270102C01093C6
:1007C0002701809164049091650462E370E0E0D4B5
:1007D00084E190E0EC01C61BD70BEAF0C632D105EC
:1007E00014F555DCBE01660F771F660F771F660F85
:1007F000771F6C1B7D0B45E150E0C50137DC64972A
:1008000039F047E050E06CE870E080ED93E02EDCDA
:100810001092E2037FCE3BDC45E150E060E070E007
:10082000C50124DCEECF33DC45E150E063E071E04C
:10083000C5011CDCE6CF1093170157CF4091ED03A3
:100840005091EE03CA018497079708F003C1CA01CB
:1008500082959295907F9827807F9827BC016F554D
:100860007F4FCA01880F991F880F991F880F991F02
:10087000840F951F9C01285C3D4F86B5883CE8F3AA
:1008800016BC81E08DBD209A80911001F901E80F1E
:10089000F11D80818EBD0DB407FEFDCF8091110149
:1008A000F901E80FF11D80818EBD0DB407FEFDCF6B
:1008B00080911201F901E80FF11D80818EBD0DB408
:1008C00007FEFDCF80911301F901E80FF11D808132
:1008D0008EBD0DB407FEFDCF80911401F901E80F24
:1008E000F11D80818EBD0DB407FEFDCF80911501F5
:1008F000F901E80FF11D80818EBD0DB407FEFDCF1B
:1009000080911601F901E80FF11D80818EBD0DB4B3
:1009100007FEFDCF80911701F901E80FF11D8081DD
:100920008EBD0DB407FEFDCF209816BC86B5803570
:10093000E8F316BC1DBC209A80910B01F901E80F69
:10094000F11D80818EBD0DB407FEFDCF80910C019D
:10095000FB01E80FF11D80818EBD0DB407FEFDCFB8
:1009600080910D01FB01E80FF11D80818EBD0DB45A
:1009700007FEFDCF80910E01FB01E80FF11D808184
:100980008EBD0DB407FEFDCF80910F01F901E80F78
:10099000F11D80818EBD0DB407FEFDCF209886B578
:1009A0008A3FE8F316BC86B58634E8F381E08DBD56
:1009B000209A80912001F901E80FF11D80818EBD00
:1009C0000DB407FEFDCF80912101F901E80FF11D63
:1009D00080818EBD0DB407FEFDCF80912201F9010B
:1009E000E80FF11D80818EBD0DB407FEFDCF809113
:1009F0002301F901E80FF11D80818EBD0DB407FEC2
:100A0000FDCF80912401F901E80FF11D80818EBD99
:100A10000DB407FEFDCF80912501F901E80FF11D0E
:100A200080818EBD0DB407FEFDCF80912601F901B6
:100A3000E80FF11D80818EBD0DB407FEFDCF8091C2
:100A40002701F901E80FF11D80818EBD0DB407FE6D
:100A5000FDCF2098CA018D97079708F0D4C0CA012E
:100A6000880F991F840F951F9C01220F331F220F9F
:100A7000331F220F331F820F931FBC01605B724034
:100A8000CA0182959295907F9827807F98279C0134
:100A90002F5E3F4F86B5883CE8F316BC81E08DBDE4
:100AA000209A80911801FB01E80FF11D80818EBD15
:100AB0000DB407FEFDCF80911901F901E80FF11D7A
:100AC00080818EBD0DB407FEFDCF80911A01FB0120
:100AD000E80FF11D80818EBD0DB407FEFDCF809122
:100AE0001B01F901E80FF11D80818EBD0DB407FED9
:100AF000FDCF80911C01F901E80FF11D80818EBDB1
:100B00000DB407FEFDCF80911D01F901E80FF11D25
:100B100080818EBD0DB407FEFDCF80911E01F901CD
:100B2000E80FF11D80818EBD0DB407FEFDCF8091D1
:100B30001F01FB01E80FF11D80818EBD0DB407FE82
:100B4000FDCF209816BC86B58035E8F316BC86B577
:100B50008A3FE8F316BC86B58634E8F316BC81E01C
:100B60008DBD209A80912801FB01E80FF11D808145
:100B70008EBD0DB407FEFDCF80912901FB01E80F6A
:100B8000F11D80818EBD0DB407FEFDCF80912A013D
:100B9000F901E80FF11D80818EBD0DB407FEFDCF78
:100BA00080912B01FB01E80FF11D80818EBD0DB4FA
:100BB00007FEFDCF80912C01F901E80FF11D808126
:100BC0008EBD0DB407FEFDCF80912D01F901E80F18
:100BD000F11D80818EBD0DB407FEFDCF80912E01E9
:100BE000F901E80FF11D80818EBD0DB407FEFDCF28
:100BF00080912F01F901E80FF11D80818EBD0DB4A8
:100C000007FEFDCF2098CA01CD97079708F09CC03A
:100C10008091D903882309F497C08091D803882351
:100C200009F492C0CA01880F991F840F951F9C0177
:100C3000220F331F220F331F220F331F820F931FE8
:100C40009C012056344086B5883CE8F316BC86B536
:100C50008A3FE8F381E08DBDF901E05CFF4F8081C0
:100C60008EBD0DB407FEFDCFF901E05CFF4F808122
:100C70008EBD0DB407FEFDCFF901E45BFF4F80810F
:100C80008EBD0DB407FEFDCFF901E15BFF4F808102
:100C90008EBD0DB407FEFDCFF901E95AFF4F8081EB
:100CA0008EBD0DB407FEFDCFF901E05CFF4F8081E2
:100CB0008EBD0DB407FEFDCFF901EE5BFF4F8081C5
:100CC0008EBD0DB407FEFDCFF901EF5BFF4F8081B4
:100CD0008EBD0DB407FEFDCFF901EC5AFF4F8081A8
:100CE0008EBD0DB407FEFDCFF901EC5AFF4F808198
:100CF0008EBD0DB407FEFDCFF901EB5BFF4F808188
:100D00008EBD0DB407FEFDCFF901EE5AFF4F808175
:100D10008EBD0DB407FEFDCFF901E75AFF4F80816C
:100D20008EBD0DB407FEFDCFF901E05CFF4F808161
:100D30008EBD0DB407FEFDCFF901E05CFF4F808151
:100D40008EBD0DB407FEFDCFCA0181559040893A92
:100D5000910520F486B5883CE8F316BCCA018B5A8D
:100D60009040079708F04DC0CA0182959295907FF8
:100D70009827807F98279C012F5C374086B58A3062
:100D8000E8F381E08DBD209A80913001F901E80FF0
:100D9000F11D80818EBD0DB407FEFDCF8091310124
:100DA000F901E80FF11D80818EBD0DB407FEFDCF66
:100DB00080913201F901E80FF11D80818EBD0DB4E3
:100DC00007FEFDCF80913301F901E80FF11D80810D
:100DD0008EBD0DB407FEFDCF80913401F901E80FFF
:100DE000F11D80818EBD0DB407FEFDCF80913501D0
:100DF000F901E80FF11D80818EBD0DB407FEFDCF16
:100E00002098443B5105B0F08091DC039091DD03C4
:100E10008D549F4F4817590768F48091DF0388234A
:100E200049F086B58233E8F3809136018EBD0DB46A
:100E300007FEFDCF4091ED035091EE032091DC03BE
:100E40003091DD0389EA90E0821B930B84179507AC
:100E500080F4493A510568F48091DE03882349F013
:100E600086B58233E8F3809136018EBD0DB407FE5E
:100E7000FDCF0000CA018B5590408F39910508F0D5
:100E800084C080910001813009F07FC086B58A3F1F
:100E9000E8F316BCCA018A559040969587959695B9
:100EA0008795FC01EE0FFF1FEE0FFF1FEE0FFF1FD8
:100EB000E81BF90B87E391E0DF01A80FB91F4C9104
:100EC0003196DF01A80FB91F3C913196DF01A80FC1
:100ED000B91F5C913196DF01A80FB91F6C91319653
:100EE000DF01A80FB91FAC913196E80FF91F70818F
:100EF000918186B58431E8F380910101882311F452
:100F000020E002C0209A20E0842F880F880F847090
:100F100085B946952F5F2830B9F7832F880F880F42
:100F2000847085B936952F5F2031B9F7852F880FEA
:100F3000880F847085B956952F5F2831B9F7862FB1
:100F4000880F880F847085B966952F5F2032B9F7B6
:100F50008A2F880F880F847085B9A6952F5F283255
:100F6000B9F7872F880F880F847085B976952F5F22
:100F70002033B9F7892F880F880F847085B996952B
:100F80002F5F2833B9F715B820982091ED033091E1
:100F9000EE03C9018D529140079708F0A2C081E08D
:100FA0008DBDC901880F991F820F931F9C01220FCD
:100FB000331F220F331F220F331F820F931F9C01F9
:100FC000205B3D4186B5883CE8F3F901ED5BFF4FBE
:100FD00080818EBD0DB407FEFDCFF901E05CFF4FAF
:100FE00080818EBD0DB407FEFDCFF901E95BFF4F97
:100FF00080818EBD0DB407FEFDCFF901EB5AFF4F86
:1010000080818EBD0DB407FEFDCFF901E25BFF4F7D
:1010100080818EBD0DB407FEFDCFF901EC5AFF4F64
:1010200080818EBD0DB407FEFDCFF901EB5BFF4F54
:1010300080818EBD0DB407FEFDCFF901EE5AFF4F42
:1010400080818EBD0DB407FEFDCFF901E05CFF4F3E
:1010500080818EBD0DB407FEFDCFF901E45BFF4F2B
:1010600080818EBD0DB407FEFDCFF901E15BFF4F1E
:1010700080818EBD0DB407FEFDCFF901E95BFF4F06
:1010800080818EBD0DB407FEFDCFF901EB5BFF4FF4
:1010900080818EBD0DB407FEFDCFF901E35BFF4FEC
:1010A00080818EBD0DB407FEFDCFF901EF5BFF4FD0
:1010B00080818EBD0DB407FEFDCFF901E25BFF4FCD
:1010C00080818EBD0DB407FEFDCFF901E25BFF4FBD
:1010D00080818EBD0DB407FEFDCF16BC86B5823073
:1010E000E8F308951F920F920FB60F9211242F93D9
:1010F0003F934F935F936F937F938F939F93AF93A0
:10110000BF93EF93FF9316BC8091ED039091EE0394
:1011100001969093EE038093ED0390DBFF91EF91A6
:10112000BF91AF919F918F917F916F915F914F91FF
:101130003F912F910F900FBE0F901F9018951F9207
:101140000F920FB60F9211248F931092EE0310920C
:10115000ED038091DA038F5F8093DA038F910F9014
:101160000FBE0F901F901895AA1BBB1B51E107C023
:10117000AA1FBB1FA617B70710F0A61BB70B881F27
:10118000991F5A95A9F780959095BC01CD010895B6
:1011900097FB092E07260AD077FD04D0E5DF06D09D
:1011A00000201AF4709561957F4F0895F6F7909599
:0811B00081959F4F0895FFCFC8
:1011B8000101545844014052584401023030300370
:1011C8000808080808080808553A4030302E3056F4
:1011D800080808080808080852583A403130302FE3
:1011E8002B3030303030FE000000000000000000DE
:1011F80000000000000000000000000000000000E7
:10120800000000005500FF00FF0000FF00FF00FF86
:101218000000FF00FF00FF0000FF00FF00FF0000CC
:10122800FF00FF00FF0000FF00FF00FF0000FF00BD
:10123800FF00FF0000FF00FF00FF0000FF00FF00AD
:10124800FF0000FF00FF00FF0000FF00FF00FF009D
:1012580000FF00FF00FF00FF00FF00FF00FFFF008E
:10126800FF00FF00FFFF00FF00FF00FFFF00FF007F
:10127800FF00FFFF00FF00FF00FFFF00FF00FF006F
:10128800FFFF00FF00FF00FFFF00FF00FF00FFFF60
:1012980000FF00FF00FFFF00FF00FF00FFFF00FF4F
:1012A80000FF00FFFF00FF00FF00FFFF00FF00FF3F
:1012B80000FFFF00FF00FF00FFFF00FF00FF00FF2F
:1012C800FF00FF00FF00FFFF00FF00FF00FFFF001F
:1012D800FF00FF00FFFF00FF00FF00FFFF00FF000F
:1012E800FF00FFFF00FF00FF0055FF00FF00FF00A9
:1012F800AAFF00FF00FF0055FF00FF00FF00AA0043
:10130800187C3C787E7E3C427C7E424082823C7CDB
:101318003C7C3C7C4242828282FE00244242444021
:1013280040424210084440C6C24242424242104231
:101338004282444404004242404240404042100835
:101348004840AAA2424242424010424292282808FB
:1013580000427C40427C7C4E7E1008704092924253
:101368007C427C3C10422492101010007E42404285
:101378004040424210084840828A42404C4802108D
:1013880042249228102000424242444040424210E7
:1013980048447E828642404644421042246C4410AF
:1013A8004000427C3C787E403C427C30427E8282D7
:1013B8003C4032423C103C186C8210FE0000000099
:1013C800307C107C7C1CFE7CFE7C7C0010000000C5
:1013D80044823082822480800282821010000000C1
:1013E8004482100202448080048282007C007C00D7
:1013F8003082100C1C847CFC087C7E0010180000D5
:101408000082103002FE02821082040010180018B8
:1014180000821040820482821082081000000018A6
:10142800007C38FE7C047C7C107C3000FEFE18308A
:101438000080A0A8AAFE8238380080A0A8AAFE8250
:10144800783C0080A0A8AAFE82FEFE0080A0A8AA80
:10145800FE827E3C0080A0A8AAFE8238380080A0C8
:10146800A8AAFEFE18300080A0A8AA000000180054
:101478000000FFFFFF24FFFFFF000000180000002E
:08148800AAAAAAFF5555550060
:00000001FF
